:020000040800F2
:100000000004022001020008910F0008950F00086B
:10001000E90F0008950F0008BD0F00080302000853
:100020000302000803020008030200085129000827
:10003000030200080302000803020008030200088C
:10004000030200080302000803020008030200087C
:1000500003020008030200083D3A0008693A00085C
:10006000953A0008C13A0008ED3A0008030200087A
:10007000030200080302000803020008030200084C
:10008000030200080302000803020008030200083C
:10009000030200080302000803020008193B0008DD
:1000A000030200080302000803020008030200081C
:1000B0006138000803020008030200080302000878
:1000C00003020008030200080302000803020008FC
:1000D00003020008030200088D1100080302000853
:1000E000813B000803020008030200080302000825
:1000F00003020008030200080302000803020008CC
:1001000003020008030200080302000803020008BB
:1001100003020008030200080302000803020008AB
:10012000030200080302000803020008030200089B
:10013000030200080302000803020008030200088B
:10014000030200080302000803020008BD30000893
:10015000030200080302000803020008030200086B
:10016000030200080302000803020008030200085B
:10017000030200080302000803020008030200084B
:100180000302000803020008A1110008030200088E
:10019000030200080302000803020008030200082B
:1001A000030200080302000803020008030200081B
:1001B000030200080302000803020008030200080B
:1001C00003020008030200080302000803020008FB
:1001D00003020008030200080302000803020008EB
:1001E00003020008030200080302000803020008DB
:1001F00003020008030200080302000803020008CB
:1002000002E000F000F8FEE772B6394880F3088893
:10021000384880F3098838484EF60851CEF200017C
:10022000086040F20000CCF200004EF63471CEF2CD
:1002300000010860BFF34F8FBFF36F8F40F20000E3
:10024000C0F2F0004EF68851CEF200010860BFF314
:100250004F8FBFF36F8F4FF00000E1EE100A4EF6A4
:100260003C71CEF200010860062080F31488BFF3D1
:100270006F8F02F0ABFB03F07BFA4FF055301F4954
:100280001B4A91423CBF41F8040BFAE71C49194A4A
:1002900091423CBF41F8040BFAE71A491A4A1B4B3A
:1002A0009A423EBF51F8040B42F8040BF8E70020D5
:1002B0001749184A91423CBF41F8040BFAE702F093
:1002C000C9FB03F0BFFA144C144DAC4203DA54F8E6
:1002D000041B8847F9E700F03FF8114C114DAC4280
:1002E00003DA54F8041B8847F9E702F0B1BB0000B9
:1002F0000004022000240220000000080000022068
:1003000000040220F03F00080024022050240220B4
:100310005024022044390220000200080002000894
:1003200000020008000200082DE9F04F2DED108AB0
:10033000C1F80CD0D0F80CD0BDEC108ABDE8F08F1D
:10034000002383F311882846A047002001F088FF8E
:1003500001F0A6FE00DFFEE770B532231F4C00253A
:100360006FF07F0623701F236570A570E5702571FF
:100370006571A571E57125726672A372E57200F070
:10038000DDFC20B10F2325726672A372E57202F0C4
:10039000A1FA044602F0D6FA0546D0B9104B9C42A9
:1003A00019D001339C4241F2883412BF0546002423
:1003B0000125002002F098FA0DB100F05BF800F082
:1003C00087FD00F001FC204600F0F4F800F052F840
:1003D000F9E70024EDE70446EBE700BF50240220D4
:1003E000010007B008B500F06DFBA0F120035842F2
:1003F000584108BD054B07B51B88022101A8ADF87F
:10040000043000F0CBFB03B05DF804FB683C00084F
:1004100010B5202383F311881248C3680BB101F093
:10042000A5FF0023104A4FF47A710E4801F062FFD5
:10043000002383F311880D4C236813B12368013B1B
:100440002360636813B16368013B6360084B1B78EA
:1004500033B9636823B9022000F0A2FC3223636041
:1004600010BD00BF5C240220110400087825022082
:1004700070240220454B46492DE9F04153F8042FE2
:10048000013201D1BDE8F0818B42F7D1414C424BA2
:1004900022689A4278D9414B9B6803F1006303F5C7
:1004A00000439A4270D2002000F0A8FB02203C4B8F
:1004B000187000F069FC3B4B1A6C00221A64196E2C
:1004C0001A66196E596C5A64596E5A66596E596992
:1004D00041F080015961596921F0800159615969E0
:1004E000196941F000511961196921F00051196130
:1004F0001B6972B62C4B2D490B601D682468BFF335
:100500004F8FBFF36F8F2A4BC3F88420BFF34F8FF9
:100510005A6922F480325A61BFF34F8FD3F880209A
:1005200043F6E07EC2F3C906C2F34E32B70752016A
:1005300002EA0E0838463146013948EA000C00F15B
:100540004040B1F1FF3FC3F874C2F5D1203A12F137
:10055000200FEDD1BFF34F8FBFF36F8FBFF34F8FDE
:10056000BFF36F8F5A6922F400325A610022C3F838
:100570005022BFF34F8FBFF36F8F202383F3118877
:10058000AD4685F308882047BDE8F081FC7F000870
:100590001C80000804800008FF7F0008502402200F
:1005A00070240220003802400080000808ED00E0BE
:1005B00000ED00E02DE9F04F99B0B34C2022FF216F
:1005C000019010A8A66800F025FCB04AA346137855
:1005D000A3B90121AE481170C360202383F31188B1
:1005E000C3680BB101F0C2FE0023AA4A4FF47A712E
:1005F000A74801F07FFE002383F31188019B13B10C
:10060000A54B019A1A600023A44AA349019F994669
:100610001C461D46984613704B600292012000F064
:10062000B3FB002F00F012829B4B1B68002B40F0A5
:100630000D8219B0BDE8F08F0220FFF7D3FE00282D
:1006400040F0FB81019BB9F1000F08BF1F46944B9E
:100650001B8802210BA8ADF82C3000F09FFADDE7D3
:100660004FF47A7000F02EFA031E0393EADB0220A7
:10067000FFF7B8FE82460028E4D0039B581E0428EA
:1006800000F2DD81DFE800F0030E1114170018A856
:100690000523042140F8343D00F080FA54464FF021
:1006A000000856E004217848F6E704217D48F3E786
:1006B00004217D48F0E71C242046043400F0A0FA11
:1006C00004210B900BA800F069FA2C2CF4D1E5E77B
:1006D000002DB7D0002CB5D00220FFF783FE0546D1
:1006E000002800F0AF8101206C4C00F087FA4FF039
:1006F00000090220207000F047FB5FFA89FA50469B
:1007000000F08CFA074658B1504609F1010900F093
:1007100095FA0028F1D12C46A9460027634B97E7AC
:1007200001233E460220237000F020FBDBF8083056
:100730009E4206D2304600F063FA0130EBD1043617
:10074000F4E70026029BA9462C461E703746524B02
:100750005E6000F0B3FB15B1002C18BF0027FFF757
:1007600049FE5BE7002D3FF46DAF002C3FF46AAF0C
:100770000220029B187000F007FB322000F0A2F963
:10078000B0F1000AC0F25E811AF0030540F05A8110
:1007900006EB0A03DBF80820934200F25381BAF516
:1007A000807F00F24F8155450DDA4FF47A7000F0EA
:1007B00089F90490049B002BC0F24481049B3C4ABD
:1007C000AB540135EFE7C820FFF70CFE05460028C3
:1007D00000F038811F2E11D8C6F1200410AB26F08E
:1007E000030033495445184428BF5446224600F0BC
:1007F000E9FA2246FF212E4800F00CFB4FEAAA0A34
:100800002B4930465FFA8AF200F00CFB04460028C0
:1008100000F01A8106EB8A0605469AE70220FFF7E8
:10082000E1FD00283FF40EAF00F02EFA00283FF45F
:1008300009AF4FF0000A5346DBF8082092451CD25E
:10084000BAF11F0F12D8109A01320FD02AF003020A
:1008500018A90A4452F8202C0B92184604220BA91E
:100860000AF1040A00F0D4FB0346E5E7504603937F
:1008700000F0C6F9039B0B90EFE718A8042140F89D
:100880004C3D00F08BF964E75024022074250220CF
:100890005C24022011040008782502207024022024
:1008A0006A3C000854240220582402206C3C0008B2
:1008B0007424022018A80023642140F8343D00F07D
:1008C00039F900287FF4BEAE0220FFF78BFD002827
:1008D0003FF4B8AE0B9800F0C3F918AB43F8480DDD
:1008E00004211846CDE718A80023642140F8343DC0
:1008F00000F020F900287FF4A5AE0220FFF772FD7A
:1009000000283FF49FAE0B9800F0B8F918AB43F8FD
:10091000440DE5E70220FFF765FD00283FF492AEA5
:1009200000F0C2F918AB43F8400DD9E70220FFF7F9
:1009300059FD00283FF486AE0BA9142000F0BAF947
:10094000824618A8042140F83CAD00F027F9514632
:100950000BA896E7322000F0B5F8B0F1000AFFF6D8
:1009600071AE1AF0030F7FF46DAE0AEB0803DBF8EB
:10097000082093423FF666AE0220FFF733FD0028C1
:100980003FF460AE2AF0030AC244D0453FF4E1AE22
:10099000404608F1040800F033F904210A900AA83F
:1009A00000F0FCF8F1E74FF47A70FFF71BFD002828
:1009B0003FF448AE00F068F900283FF4AFAE109B5A
:1009C00001330CD0082210A9002000F02BFA0028D7
:1009D0003FF4A4AE2022FF2110A800F01BFAFFF77D
:1009E00009FD374801F042FC23E6002D3FF42AAE12
:1009F000002C3FF427AE18A80023642140F8343DB2
:100A000000F098F8824600287FF41CAE0220FFF721
:100A1000E9FC00283FF416AE0390FFF7EBFC41F22F
:100A20008830574601F022FC0B9800F091FA00F054
:100A300045FA039B1C461D46F0E5054689E64FF046
:100A40000008FFE52546FDE52C4667E6002000F09E
:100A500039F80490049B002BFFF6E3AD012000F071
:100A600085F9049B213B122B3FF6D8AD01A252F829
:100A700023F000BF3906000861060008D10600080F
:100A80001D0600081D0600081D0600086507000871
:100A9000550900081D080008B5080008E708000807
:100AA000150900081D0600082D0900081D0600088C
:100AB000A7090008530700081D060008EB090008F5
:100AC000A08601002DE9F3474FF47A75002402AEA9
:100AD000154F4543DFF8588006F8014D97F900306F
:100AE0005FFA84F95A1C01D0A34212D158F82400AD
:100AF000012231460368D3F820A02B46D0470128B5
:100B000007D10A4B9DF8070083F8009002B0BDE8BA
:100B1000F0870134032CE1D14FF4FA7001F0A6FB09
:100B20004FF0FF30F2E700BF00240220C42502206E
:100B3000783C00082DE9F0474FF47A75064600240A
:100B4000134F4D43DFF8508097F900305FFA84F976
:100B50005A1C01D0A34210D158F824000422314677
:100B60000368D3F820A02B46D047042805D1094BB1
:100B7000002083F80090BDE8F0870134032CE3D116
:100B80004FF4FA7001F072FB4FF0FF30BDE8F087D0
:100B900000240220C4250220783C0008074B30B412
:100BA0001A78074B53F822400A460146236820462C
:100BB000DD69044BAC4630BC604700BFC425022051
:100BC000783C0008A086010070B50A4C00250A4E4A
:100BD00001F086FD207030682378834208D901F047
:100BE00079FD336805440133B5F5004F3360F2D326
:100BF00070BD00BFC52502208025022001F01CBE6B
:100C000000F1006000F500400068704700F10060EE
:100C1000920000F5004001F0A9BD0000054B1A68E4
:100C2000054B1B789B1A834202D9104401F052BD38
:100C30000020704780250220C525022038B5074DC9
:100C400004462868204401F04DFD28B92868204456
:100C5000BDE8384001F05EBD38BD00BF80250220F0
:100C600010F0030308D1B0F5806F05D800F10050F3
:100C7000A0F571200068704700207047014BC058F4
:100C8000704700BF20F4F01F064991F8243033B1BB
:100C900000230822086A81F82430FFF7B7BF01203B
:100CA000704700BF84250220014B1868704700BFC1
:100CB000002004E01F4BF0B51E681F4BC6F30B026B
:100CC000360C1F885D68BA4293F9084022D09F898C
:100CD000BA4221D01F8BBA4206D102220C2404FB57
:100CE00002335D6893F90840B6F5805F16D041F293
:100CF00001039E4208BF5A24421E013D0B460A448E
:100D0000934215D215F9016F581C4EB1034600F8F5
:100D1000016CF5E70022E1E70122DFE74124EBE780
:100D20002C2582421D7001D9981C5C70401AF0BDC0
:100D30001846FBE7002004E004240220094B5B88EE
:100D4000B3F5805F09D041F20102934207D101223D
:100D5000054B03EB8203D87870470022F8E70020A8
:100D6000704700BF002004E0703C0008022804D156
:100D70004FF48002034B9A6170470128FCD14FF475
:100D80000002F7E700080240022803D14022034B8B
:100D90009A6170470128FCD18022F8E700080240E0
:100DA000022805D1064A536983F040035361704716
:100DB0000128FCD1024A536983F08003F6E700BFA3
:100DC00000080240002310B5934203D0CC5CC45409
:100DD0000133F9E710BD000030B5441E14F9010FCE
:100DE0000B4658B193F900500131854206D11AB92A
:100DF00093F90020801A30BD013AEFE7002AF7D1BD
:100E0000104630BD02460346981A13F9011B00290B
:100E1000FAD1704702440346934202D003F8011B03
:100E2000FAE770472DE9F047234C054688461746F8
:100E300094F8243083BB2E46DFF87C90C7B394F837
:100E400024302BB92022FF2148462662FFF7E2FF1B
:100E500094F824004146C0F1080504EB8000BD422F
:100E600028BF3D465FFA85FAAD00A7EB0A072A4680
:100E70002E44FFF7A7FF94F82430A844FFB29A4409
:100E80005FFA8AFABAF1080F84F824A0D6D1FFF7E6
:100E9000FBFE0028D2D108E0266A06EB8306B042AA
:100EA000CAD0FFF7F1FE0028C5D10020BDE8F087C9
:100EB0000120BDE8F08700BF84250220024B1A788C
:100EC000024B1A70704700BFC42502200024022084
:100ED00038B5184C184D204600F076FC29462046BF
:100EE00000F09EFC2D681548EA6ED2F8043843F0F5
:100EF0000203C2F8043801F0B9F91149284600F09C
:100F00009DFDEA6E0F48D2F804380F49A04223F045
:100F10000203C2F804384FF4E1330B6001D000F053
:100F2000B1FB0A48A04204D00749BDE8384000F0B0
:100F3000A9BB38BD58310220943D000840420F0043
:100F4000B83D000848260220AC250220B426022025
:100F500038B50B4B05461A780A4B53F822400A4B1A
:100F60009C420CD0094B002118221846FFF752FF73
:100F7000056001462046BDE8384000F083BB38BD1F
:100F8000C4250220783C000858310220AC250220FC
:100F9000FEE7000000B59BB0EFF3098168226846C8
:100FA000FFF710FFEFF30583034B9A6B9A6A9A6A77
:100FB0009A6A9A6A9B6AFEE700ED00E000B59BB072
:100FC000EFF3098168226846FFF7FCFEEFF3058323
:100FD000044B9A6B9A6A9A6A9A6A9A6A9A6A9B6AA4
:100FE000FEE700BF00ED00E000B59BB0EFF3098124
:100FF00068226846FFF7E6FEEFF30583034B5A6B62
:101000009A6A9A6A9A6A9A6A9B6AFEE700ED00E019
:1010100030B50A44074D91420BD011F8013B092429
:101020005840013CF7D040F300032B4083EA5000C6
:10103000F7E730BD2083B8ED002304491A465A5023
:10104000C81808334260802BF9D17047C8250220A8
:10105000026843681143016003B1184770470000FC
:10106000024A136843F0C003136070470044004015
:10107000024A136843F0C0031360704700780040D1
:101080002DE9F047C66D05463768F46920073462DC
:101090001AD014F0080F0CBF00218021E20748BFCE
:1010A00041F02001A3074FF0200348BF41F0400169
:1010B000600748BF41F4807183F31188281DFFF752
:1010C000C7FF002383F31188E2050AD5202383F3A9
:1010D00011884FF40071281DFFF7BAFF002383F336
:1010E00011884FF020094FF0000A14F0200831D188
:1010F0003B0616D54FF0200905F1380A200610D519
:1011000089F31188504600F031FA00282FDA0821BF
:10111000281DFFF79DFF27F080033360002383F332
:10112000118879060DD562060BD5202383F311882B
:10113000EA6C2B6D9A4201D12B6CEBB9002383F33F
:101140001188E30620D5AA6E1369EBB15069BDE89A
:10115000F047184789F31188736A284695F8641098
:10116000194000F09DFA8AF31188F469BDE7B06276
:1011700088F31188F469C1E727F040071021281D82
:10118000FFF766FF3760D9E7BDE8F08708B5034889
:10119000FFF776FFBDE8084001F0EABB48260220D1
:1011A00008B50348FFF76CFFBDE8084001F0E0BB5D
:1011B000B426022037B51F4C1F4D204600F056FACA
:1011C000009404F1140000234FF400721B4900F056
:1011D00017F94FF40072009404F13800184B1949C4
:1011E00000F090F9184B25660B21E3652620174C7B
:1011F00000F090F8204600F039FA04F11400009451
:1012000000234FF40072124900F0FAF804F138009C
:1012100000944FF400720F4B0F4900F073F90F4B1D
:101220000B215220E365256603B0BDE8304000F095
:1012300071B800BF4826022080F93703202702201A
:1012400061100008202B022000440040B426022038
:101250002029022071100008202D02200078004073
:10126000284B002908BF1946037C012B816630B545
:101270000CD1254B984235D1244B1A6C42F40032E4
:101280001A641A6E42F400321A661B6E0A68036E04
:10129000C46D03EB5203B3FBF2F34A68150442BF7B
:1012A00023F0070503F0070343EA4503E3608B6877
:1012B00043F040036360CB68510543F00103A36032
:1012C00042F4967343F0010323604FF0FF3323622F
:1012D00005D512F0102211D0B2F1805F10D080F845
:1012E000643030BD0A4B9842D0D1084B1A6C42F0A2
:1012F00080421A641A6E42F08042C5E77F23EEE70F
:101300003F23ECE7B03C00084826022000380240AA
:10131000B426022000F1604300F01F0209014009D9
:1013200003F56143C9B2800083F80013012300F183
:101330006040934000F56140C0F880310360704721
:10134000F8B51546826804460B46AA4200D2856865
:10135000A1692669761AB54207D218462A46FFF7D0
:1013600031FDA3692B44A3610DE011D9AF1B3246B7
:101370001846FFF727FD3A46E1683044FFF722FDA3
:10138000E2683A44A261A36828465B1BA360F8BDEB
:1013900018462A46FFF716FDE368E4E783689342A0
:1013A0002DE9F04104460F46154600D28568606974
:1013B0002669361AB54207D22A463946FFF702FD9A
:1013C00063692B4463610EE013D9A5EB060832462E
:1013D0003946FFF7F7FC4246B919E068FFF7F2FC1F
:1013E000E26842446261A36828465B1BA360BDE8D3
:1013F000F0812A463946FFF7E5FCE368E2E70000A2
:1014000010B50A440024C361029B00604060846000
:10141000C160816141610261036210BD08B58269EA
:101420004369934201D1826882B982680132826045
:101430005A1C42611970426903699A4201D3C36818
:101440004361002100F02EFF002008BD4FF0FF3067
:1014500008BD000070B5202304460E4683F31188B2
:10146000A568A5B1A368A269013BA360531CA36151
:1014700015782269934224BFE368A361E3690BB145
:1014800020469847002383F31188284670BD3146D3
:10149000204600F0F7FE0028E2DA85F3118870BDDF
:1014A0002DE9F74F05460F4690469A46D0F81C9016
:1014B000202686F311884FF0000B144664B12246B3
:1014C00039462846FFF73CFF034668B9514628468F
:1014D00000F0D8FE0028F1D0002383F31188A8EB98
:1014E000040003B0BDE8F08FB9F1000F03D0019004
:1014F0002846C847019B8BF31188E41A1F4486F3E2
:101500001188DBE7C160816141611144C361009BC7
:10151000006040608260016103627047F8B5044674
:101520000E461746202383F31188A568A5B1A3684A
:10153000013BA36063695A1C62611E702369626982
:101540009A4224BFE3686361E3690BB12046984780
:10155000002080F31188F8BD3946204600F092FE45
:101560000028E2DA85F31188F8BD0000836942693A
:101570009A4210B501D182687AB9826801328260DC
:101580005A1C82611C7803699A4201D3C368836143
:10159000002100F087FE204610BD4FF0FF3010BD47
:1015A0002DE9F74F05460F4690469A46D0F81C9015
:1015B000202686F311884FF0000B144664B12246B2
:1015C00039462846FFF7EAFE034668B951462846E1
:1015D00000F058FE0028F1D0002383F31188A8EB17
:1015E000040003B0BDE8F08FB9F1000F03D0019003
:1015F0002846C847019B8BF31188E41A1F4486F3E1
:101600001188DBE7026843681143016003B11847A2
:10161000704700001430FFF743BF00004FF0FF3366
:101620001430FFF73DBF00003830FFF7B9BF0000AE
:101630004FF0FF333830FFF7B3BF00001430FFF72F
:1016400009BF00004FF0FF311430FFF703BF000067
:101650003830FFF763BF00004FF0FF323830FFF73C
:101660005DBF000000207047FFF7A4BD044B03607E
:10167000002343608360C36001230374704700BF8D
:10168000C83C000810B52023044683F31188FFF7F7
:10169000E7FD02232374002383F3118810BD0000AB
:1016A00038B5C36904460D461BB904210844FFF749
:1016B000A9FF294604F11400FFF7B0FE002806DA5E
:1016C000201D4FF48061BDE83840FFF79BBF38BD57
:1016D000026843681143016003B118477047000076
:1016E00013B5446BD4F894341A681178042915D1D1
:1016F000217C022912D11979012312898B401342CE
:101700000CD101A904F14C0001F03AFFD4F8944443
:101710000246019B2179206800F0E0F902B010BD7B
:10172000143001F0BDBE00004FF0FF33143001F063
:10173000B7BE00004C3001F08FBF00004FF0FF3308
:101740004C3001F089BF0000143001F08BBE000066
:101750004FF0FF31143001F085BE00004C3001F035
:101760005BBF00004FF0FF324C3001F055BF00006E
:10177000D0F8942438B5136805461978042901D0A7
:10178000012038BD017C0229FAD1127901205C893F
:1017900090400440F4D105F1140001F01DFE024612
:1017A0000028EDD0D5F894544FF4807328686979F7
:1017B00000F082F9204638BD406BFFF7D9BF00002A
:1017C00000207047704700007FB5124B01250226AC
:1017D000044603600023057400F184024360294637
:1017E0008360C3600C4B0290143001934FF48073FC
:1017F000009601F0CDFD094B04F5237229460193B3
:1018000004F14C004FF480730294009601F094FEB2
:1018100004B070BDF03C0008B9170008E1160008DC
:101820000B68202282F311880A7903EB820210628E
:101830004A790D3243F822008A7912B103EB820310
:1018400018620223C0F894140374002383F31188F0
:101850007047000038B5037F044613B190F8543048
:10186000ABB90125201D0221FFF732FF04F114005E
:1018700025776FF0010100F021FD84F8545004F148
:101880004C006FF00101BDE8384000F017BD38BDD5
:1018900010B5012104460430FFF71AFF0023237717
:1018A00084F8543010BD000038B5044600251430CB
:1018B00001F086FD04F14C00257701F055FE201D56
:1018C00084F854500121FFF703FF2046BDE838405B
:1018D000FFF74EBF90F85C3003F06003202B19D166
:1018E00090F85D20212A0AD0222A4FF000030ED062
:1018F000202A0FD1084A02650722426504E0064B00
:101900000365072343650023836501207047036552
:101910004365F9E70020704728240220D0F894346A
:1019200037B51A680446117804291AD1017C0229B6
:1019300017D11979012312898B40134211D100F17B
:101940004C05284601F0D0FE58B101A9284601F007
:1019500017FED4F894440246019B2179206800F0D8
:10196000BDF803B030BD000000EB8103F7B51C6A81
:1019700005460E46F4B1202383F3118805EB860754
:10198000201D08214C34FFF7A3FEFB685B691B6830
:1019900013B1204601F002FE01A9204601F0F0FD3E
:1019A000024648B1019B3146284600F097F80023D3
:1019B00083F3118803B0F0BDFB685A691268002AEE
:1019C000F5D01B8A013B1340F1D105F15C02EAE737
:1019D0000D3138B550F82140DCB1202383F3118854
:1019E000D4F894241368527903EB8203DB689B6973
:1019F0005D6845B104216018FFF76AFE294604F1CD
:101A0000140001F0F3FC2046FFF7B2FE002383F33D
:101A1000118838BD7047000001F0A2B8012300F121
:101A2000240200F1380103700023436042F8043BB4
:101A30008A421361FAD103814381704738B5044665
:101A4000202383F3118800254160C560056145614D
:101A50008561C561056201F093F80223237085F367
:101A6000118838BD70B500EB8103054650690E46FC
:101A70001446DA6018B110220021FFF7CBF9A069F3
:101A800018B110220021FFF7C5F931462846BDE8FC
:101A9000704001F03FB90000028902F001020281AA
:101AA000428902F0010242810022026142618261A8
:101AB000C261026201F0C2B9F0B4012500EB8104F9
:101AC00047898D40E4683D43A46945812360002334
:101AD000A2606360F0BC01F0DDB90000F0B4012544
:101AE00000EB810407898D40E4683D43646905810A
:101AF00023600023A2606360F0BC01F057BA0000CD
:101B000070B50223002504460370A0F8645080F8E5
:101B1000665080F8675005814581C5600561456163
:101B20008561C561056280F84C5001F08FF86368EB
:101B30001B6823B129462046BDE87040184770BD98
:101B40000278436880F8682005221B6802700BB198
:101B50000421184770470000436890F868201B680C
:101B600002700BB1052118477047000090F84C3007
:101B700070B5044613B1002380F84C3004F15C02C8
:101B8000204601F07DF963689B6863BB94F85C5064
:101B900015F0600615D194F85D3005F07F0545EA33
:101BA000032540F202339D4200F00E815BD8022DE6
:101BB00000F0DC803FD8002D00F08780012D00F080
:101BC000CF800021204601F0C5FB0021204601F016
:101BD000B7FB63681B6813B10621204698470623AC
:101BE00084F84C3070BD204698470028CED094F839
:101BF000632094F8623043EA0223626D934238BF57
:101C0000636594F95C30656D002B4FF0200380F222
:101C1000FD80002D00F0EC80092284F84C2083F335
:101C200011880021636D226D2046FFF757FF0023C6
:101C300083F3118870BDB5F5817F00F0B180B5F5F3
:101C4000407F49D0B5F5807FBBD194F85E30012B41
:101C5000B7D1B4F8643023F00203A4F864302665E9
:101C60006665A665C3E740F201639D421ED8B5F5DF
:101C7000C06F3BD2B5F5A06FA3D1B4F85C30B3F51B
:101C8000A06F0ED194F85E30204684F8663001F0E3
:101C900035F863681B6813B1012120469847032378
:101CA0002370002323656365A365A0E7B5F5106F76
:101CB00032D040F602439D4252D0B5F5006F80D13C
:101CC00004F167032365012324E004F16403A5659F
:101CD0002365022363658AE794F85E30012B7FF465
:101CE00070AFB4F8643043F00203B6E794F86120B3
:101CF0002046616894F860304D6843EA022394F806
:101D00005F1094F85E20A84700283FF45AAF43685C
:101D1000236503686365A4E72378042B10D120238F
:101D200083F311882046FFF7B7FE86F311886368B6
:101D3000032184F867601B6821700BB12046984727
:101D400094F85E30002BACD084F867300423237005
:101D500063681B68002BA4D0022120469847A0E7A7
:101D6000374B23650223636500239DE794F86010D9
:101D7000204611F0800F01F00F010ED001F072F833
:101D8000012806D002287FF41CAF2E4B6065236526
:101D900067E72D4B6565236563E701F055F8EFE7CD
:101DA00094F85E30002B7FF40CAF94F8603013F0A1
:101DB0000F013FF476AF1A06204602D501F0DEFA95
:101DC0006FE701F0D1FA6CE794F85E30002B7FF4F6
:101DD000F8AE94F8603013F00F013FF462AF1B06C9
:101DE000204602D501F0B6FA5BE701F0A9FA58E700
:101DF000142284F84C2083F311882B462A46294666
:101E00002046FFF759FE85F3118870BD5DB115229C
:101E100084F84C2083F311880021636D226D2046E5
:101E2000FFF74AFE03E70B2284F84C2083F3118866
:101E30002B462A4629462046FFF750FEE3E700BF1F
:101E4000203D0008183D00081C3D000838B590F8FA
:101E50004C300446152B29D8DFE803F03E2828280B
:101E600028283E28280B29392828282828282828E7
:101E70003E3E90F8631090F86220436D42EA0122E2
:101E80009A4214D9C268128AB3FBF2F502FB1535E7
:101E90006DB9202383F311882B462A462946FFF784
:101EA0001DFE85F311880A2384F84C3038BD1423B5
:101EB00084F84C30202383F31188002320461A46EF
:101EC0001946FFF7F9FD002383F3118838BD836DB0
:101ED00003B198470023E7E7002101F03BFA002116
:101EE000204601F02DFA63681B6813B106212046D5
:101EF00098470623D8E7000090F84C20152A38B5FB
:101F0000044622D80123934040F6416213421DD17A
:101F100013F480150FD19B0217D50B2380F84C309A
:101F2000202383F311882B462A462946FFF7D6FD46
:101F300085F3118838BDC3689B695B682BB9836DD5
:101F400003B19847002384F84C3038BD002101F0DC
:101F500001FA0021204601F0F3F963681B6813B110
:101F60000621204698470623EDE70000024B002299
:101F70001B605B609A607047202F022000238268FC
:101F80000374054B1B6899689142FBD25A68036041
:101F90004260106058607047202F022008B520234F
:101FA00083F31188037C032B05D0042B0DD02BB9B0
:101FB00083F3118808BD436900221A604FF0FF3394
:101FC0004361FFF7DBFF0023F2E790E80C001A60A3
:101FD00002685360F2E70000002382680374054B37
:101FE0001B6899689142FBD85A6803604260106090
:101FF00058607047202F0220054B19690874186833
:10200000026853601A60186101230374FEF78CB9EB
:10201000202F02204B1C30B5054687B00A4C10D04B
:10202000236901A8094A00F065F92846FFF7E4FF93
:10203000049B13B101A800F099F92369586907B00E
:1020400030BDFFF7D9FFF8E7202F02209D1F0008C1
:1020500038B50C4D044641612B6981689A689142FC
:1020600003D8BDE83840FFF789BF1846FFF786FF61
:1020700001232C61014623742046BDE83840FEF759
:1020800053B900BF202F0220044B1A681B699068C7
:102090009B68984294BF002001207047202F0220A7
:1020A00010B5084C236820691A6854602260012228
:1020B00023611A74FFF790FF01462069BDE81040C4
:1020C000FEF732B9202F0220FEE7000010B5194CB0
:1020D000FFF74CFF00F000F980221749204600F07E
:1020E00085F8012344F8180C0374144B144AD9687A
:1020F00021F4E0610904090C0A431249DA60CA6854
:1021000042F08072CA60104A1049C2F8B01F1168CC
:1021100041F0010111601022DA77202283F8222099
:10212000002383F3118862B60948BDE8104000F02F
:102130007FB800BF482F0220243D000800ED00E0DA
:102140000003FA05F0ED00E0001000E055CEACC54C
:102150002C3D00082DE9F84F1E4C4FF00008656932
:1021600004F11407C1464FF08043266AAA685B6AEF
:102170009E1B96421CD34FF0200AAA68236AD5F80A
:102180000CB0B61A134423622B68BB425F606361D4
:10219000C5F80C8001D101F0D1FA89F311882869C2
:1021A000D8478AF311886569AB689E42E5D2DAE7C1
:1021B0006269BA420CD0916823628E1B9660A8684F
:1021C00002282CBF1818981CBDE8F84F01F0BCBAC3
:1021D000BDE8F88F202F0220034B59685A68521A25
:1021E0009042FBD8704700BF001000E082600222DE
:1021F00002740022427470478368A3F17C0243F8A2
:102200000C2C026943F83C2C426943F8382C074AED
:1022100043F81C2CC268A3F1180043F8102C0222CA
:1022200003F8082C002203F8072C7047410300082C
:1022300010B5202383F31188FFF7DEFF0021044649
:10224000FFF706FF002383F31188204610BD00002E
:10225000024B1B6958610F20FFF7CEBE202F0220D2
:10226000202383F31188FFF7F3BF000008B5014670
:10227000202383F311880820FFF7CCFE002383F38B
:10228000118808BD49B1064B42681B6918605A6045
:10229000136043600420FFF7BDBE4FF0FF3070476E
:1022A000202F02200368984206D01A68026050600E
:1022B00018465961FFF762BE7047000038B5044602
:1022C0000D462068844200D138BD036823605C60FD
:1022D0004561FFF753FEF4E7054B03F114025A6121
:1022E0009A614FF0FF32DA6100221A62704700BF34
:1022F000202F0220F8B503614FF08043C26002290D
:102300005C6A0646184B38BF02211A461F4652F82F
:10231000145F95420AD1586198611C62056045605E
:1023200081600819BDE8F84001F000BA186AAB688E
:10233000241A0C1902D3E41A2D6804E09C4202D23C
:10234000204401F001FAAB689C42F4D86B68356018
:1023500073601E604FF0FF336E60B460A968091BA4
:10236000A960FB61F8BD00BF202F022010B41B4CF8
:10237000234653F8141F814210D0416802680A6056
:10238000026851609A424FF00001C16003D0936827
:1023900081680B4493605DF8044B70470A68002025
:1023A0009A4262615360C86003D15DF8044B01F04A
:1023B000C5B9936888680344206A93604FF08042EF
:1023C000526A121A9342E6D9991A5DF8044B012910
:1023D00098BF931C184401F0B7B900BF202F02200A
:1023E00000207047FEE70000704700004FF0FF300C
:1023F00070470000022906D0032906D001290648AB
:1024000018BF0020704705487047032A9ABF044848
:1024100000EBC20000207047143E0008C83D0008D1
:102420003024022070B59AB006460846144601AD25
:10243000294600F095F82846FEF7E4FCC0B2431C9C
:102440005B0086E8180023700323023404F8013C83
:1024500000231946DAB20234904201D81AB070BD96
:10246000EA5C013304F8011C04F8022CF2E70000D6
:1024700008B5202383F311880348FFF74FFA0023A0
:1024800083F3118808BD00BF5831022010B50446FF
:10249000052916D8DFE801F016150316161D2023AE
:1024A00083F311880E4A0121FFF7DCFA20460D4A1A
:1024B0000221FFF7D7FA0C48FFF7F6F9002383F360
:1024C000118810BD202383F311880748FFF7C2F954
:1024D000F4E7202383F311880348FFF7D9F9EDE7E8
:1024E0004C3D0008703D00085831022038B50C4DB5
:1024F0000C4C2A460C4904F10800FFF793FF05F144
:10250000CA0204F110000949FFF78CFF05F5CA72F1
:1025100004F118000649BDE83840FFF783BF00BF4B
:1025200020360220302402209C3D0008A43D0008F3
:10253000AF3D000870B5044608460D46FEF762FC44
:10254000C6B22046013403780BB9184670BD324636
:102550002946FEF741FC0028F3D1012070BD0000A0
:102560002DE9F84F05460C46FEF74CFC2B49C6B248
:102570002846FFF7DFFF2A492846FFF7DBFF08B1AF
:102580001036F6B2632E0DD8DFF89080DFF8909009
:10259000244FDFF898A0DFF898B02E7846B926705F
:1025A000BDE8F88F29462046BDE8F84F01F054BB3E
:1025B000252E2ED1072241462846FEF70DFC70B984
:1025C000DBF800300735073444F8073CBBF804302B
:1025D00024F8033C9BF8063004F8013CDDE70822B0
:1025E00049462846FEF7F8FB98B9A21C0E4B13F893
:1025F000011F023209095345C95D02F8041C19780C
:1026000001F00F01C95D02F8031CF0D11834083540
:10261000C3E7267001350134BFE700BF343E000830
:10262000AF3D0008443E00081FF4F01F2BF4F01FDC
:102630003C3E0008BFF34F8F024AD368DB03FCD453
:10264000704700BF003C024008B5074B1B7853B9E8
:10265000FFF7F0FF054B1A69002A04DA044A5A60B2
:1026600002F188325A6008BD7E380220003C0240E8
:102670002301674508B5054B1B7833B9FFF7DAFF2F
:10268000034A136943F00043136108BD7E380220FA
:10269000003C02400B2870B513D80B4A0B4C137842
:1026A00063B94FF000610A4E44F8231056F82350E6
:1026B00001330C2B2944F7D10123137054F8200067
:1026C00070BD002070BD00BFB038022080380220ED
:1026D000583E0008014B53F820007047583E000850
:1026E0000C2070470B2810B5044601D9002010BDFE
:1026F000FFF7D0FF064B53F824301844C21A0BB929
:10270000012010BD12680132F0D1043BF6E700BF92
:10271000583E00080B2810B5044621D8FFF78AFF61
:10272000FFF792FF0F4AF323D360C300DBB243F4F9
:10273000007343F002031361136943F480331361A0
:10274000FFF778FFFFF7A6FF074B53F8241000F0C0
:10275000DBF8FFF78FFF2046BDE81040FFF7C2BF50
:10276000002010BD003C0240583E00082DE9F8430F
:1027700012F0010315463FD18218B2F1026F3BD22D
:102780002B4B1B6813F0010336D0FFF75DFF294C7C
:10279000F32340F20127E360FFF74CFF032D01D93B
:1027A000830712D00F46401A224C40F20118EB1B4F
:1027B000C6190B44012B236924D823F0010323619C
:1027C000FFF758FF0120BDE8F883236923F4407325
:1027D000236123693B43236151F8046B0660BFF317
:1027E0004F8FFFF727FF03689E4208D0236923F02D
:1027F00001032361FFF73EFF0020BDE8F883043D9D
:102800000430CBE723F44073B9462361236943EADC
:102810000803236137F8023B3380BFF34F8FFFF784
:1028200009FF3688B6B2B9F80030B342BFD0DDE751
:1028300000380240003C0240084908B50B7828B136
:1028400053B9FFF701FF01230B7008BD23B10870D6
:10285000BDE80840FFF70EBF08BD00BF7E3802206C
:1028600002440439064BD2B210B5904200D110BDDB
:10287000441C00B253F8200041F8040FE0B2F4E722
:1028800050280040104B30B51C6F240407D41C6F37
:1028900044F400741C671C6F44F400441C670B4C28
:1028A000024404392368D2B243F480732360084B96
:1028B000904200D130BD441C51F8045F00B243F88F
:1028C0002050E0B2F4E700BF003802400070004042
:1028D0005028004007B5012201A90020FFF7C0FFE2
:1028E000019803B05DF804FB13B50446FFF7F2FF4F
:1028F000A04206D002A90122002041F8044DFFF7B2
:10290000C1FF02B010BD00000144BFF34F8F064B62
:10291000884204D3BFF34F8FBFF36F8F7047C3F864
:102920005C022030F4E700BF00ED00E0034B1B68C1
:102930009B0042BF0122024B1A707047743802405C
:10294000B1380220014B1878704700BFB13802201F
:10295000064A536823F001035360EFF30983683399
:1029600083F30988002383F31188704730EF00E078
:1029700010B5202383F31188104B5B6813F40063B8
:1029800018D0F1EE103AEFF309844FF0807344F859
:102990004C3C0B4BDB6844F8083CA4F1680383F320
:1029A0000988FFF771FB18B1064B44F8503C10BD85
:1029B000054BFAE783F3118810BD00BF00ED00E07E
:1029C00030EF00E05103000854030008F0B5BFF3F6
:1029D0004F8FBFF36F8F1D4B0021C3F85012BFF311
:1029E0004F8FBFF36F8F5A6942F400325A61BFF3C1
:1029F0004F8FBFF36F8FC3F88410BFF34F8FD3F89F
:102A0000802043F6E076C2F3C904C2F34E32A50734
:102A1000520102EA060E284621464EEA0007013915
:102A200000F14040C3F860724F1CF6D1203A12F119
:102A3000200FEED1BFF34F8F5A6942F480325A61B2
:102A4000BFF34F8FBFF36F8FF0BD00BF00ED00E00D
:102A5000FEE70000084A094B09498B4204D3094AA2
:102A60000021934205D3704752F8040F43F8040B3A
:102A7000F3E743F8041BF4E73C4000084439022024
:102A80004439022044390220036F002230B5114638
:102A9000C46E9D684FF0FF3004EB42130132954243
:102AA000C3F80019C3F81019C3F80809C3F8001BCC
:102AB000C3F8101BC3F8080BEED24FF00113C4F893
:102AC0001C3830BD890141F02001016103699B067A
:102AD000FCD41220FFF780BB204B03EB80022DE9D2
:102AE000F047D2F80CE0461CDD6EDEF8142005EB52
:102AF0000636D2F800C005EB4018516861450BD38B
:102B00000123D5F8342803FA00F022EA0000C5F8C2
:102B100034081846BDE8F087ACEB0103BEF810405E
:102B2000A34228BF2346D8F81849A4B2B3EB840FB8
:102B300010D894681F46A4F1040959F804AF042F73
:102B4000C6F800A001D9043FF7E71C440B44946089
:102B50005360D2E70020BDE8F08700BFB438022000
:102B600010B5054C2046FEF759FF4FF0A043E36631
:102B7000024B236710BD00BFB4380220AC3E0008F2
:102B80000378012B70B5054650D12A4BC46E98428C
:102B90001BD1294B0E2143205A6B42F080025A630D
:102BA0005A6D42F080025A655A6D5A6942F08002AD
:102BB0005A615A6922F080025A615B69FEF7AAFBEA
:102BC0001E4BE3601E4BC4F800380023EE6EC4F8C1
:102BD000003EC02323604FF40413A3633369002B2A
:102BE000FCDA01230C203361FFF7F6FA3369DB07C7
:102BF000FCD41220FFF7F0FA3369002BFCDA002630
:102C00002846A660FFF740FF6B68C4F81068DB68D1
:102C1000C4F81468C4F81C684BB90A4BA3614FF0A0
:102C2000FF336361A36843F00103A36070BD064BEB
:102C3000F4E700BFB43802200038024040140040DE
:102C400003002002003C30C0083C30C0F8B5C46E20
:102C5000054600214FF000662046FFF733FF296F3D
:102C600000234FF001128F684FF0FF30C4F8343862
:102C7000C4F81C2804EB431201339F42C2F80069D8
:102C8000C2F8006BC2F80809C2F8080BF2D20B6850
:102C9000EA6E6B67636210231361166916F0100603
:102CA000FBD11220FFF798FAD4F8003823F4FE6322
:102CB000C4F80038A36943F4402343F01003A36130
:102CC0000923C4F81038C4F814380A4BEB604FF0ED
:102CD000C043C4F8103B084BC4F8003BC4F810696B
:102CE000C4F800396B6F03F1100243F480136A6774
:102CF000A362F8BD883E000840800010C26E90F8C4
:102D00006610D2F8003823F4FE6343EA0113C2F8D8
:102D1000003870472DE9F0410EB20D4600EB8608F1
:102D2000D8F80C100F6807F00303022B50D0032BC8
:102D300050D03D4A3D4F012B18BF1746C46E4FEA95
:102D4000451E002205F1100C04EB0E03C3F8102BF6
:102D50008A69002A40D04A8A05F158033A435B0148
:102D6000E2500123D4F81C2803FA0CF31343C4F8EF
:102D70001C38A64400234A69CEF8103905F13F03F8
:102D8000002A39D00A8A04EB8303898B920801292F
:102D900088BF4A43416F561841EA024229464667B6
:102DA00020465A60FFF78EFED8F80C301B8A43EAA3
:102DB00085531F4305F148035B01E7500123D4F815
:102DC0001C2803FA05F51543C4F81C58BDE8F0812A
:102DD000174FB3E7174FB1E704EB4613D3F8002BB7
:102DE00022F40042C3F8002B0123D4F81C2803FA74
:102DF0000CF322EA0303BAE704EB83030E4A04EB65
:102E0000461629465A602046FFF75CFED6F8003980
:102E1000012223F4004302FA05F5C6F80039D4F87C
:102E20001C3823EA0505CFE700800010008004105D
:102E30000080081000800C1000040002026F12686D
:102E40004267FFF721BE00005831C36E49015B584D
:102E500013F4004004D013F4001F14BF012002201B
:102E6000704700004831C36E49015B5813F40040BD
:102E700004D013F4001F14BF01200220704700008B
:102E800000EB8101CB68196A0B6813604B685360D3
:102E90007047000000EB810330B5DD68AA69136854
:102EA000D36019B9402B84BF402313606B8A146828
:102EB000C26E1C4402EB4110013C09B2B4FBF3F4B6
:102EC0006343033323F0030343EAC44343F0C043A3
:102ED000C0F8103B2B6803F00303012B0ED1D2F88E
:102EE000083802EB411013F4807FD0F8003B14BF88
:102EF00043F0805343F00053C0F8003B02EB411213
:102F0000D2F8003B43F00443C2F8003B30BD000060
:102F10002DE9F041244D0446EE6E06EB4013D3F844
:102F2000087B3807C3F8087B0AD5D6F81438190788
:102F300006D505EB840321462846DB685B68984785
:102F4000FA072FD5D6F81438DB072BD505EB840309
:102F5000D968CCB98B69488A5E68B6FBF0F200FB91
:102F600012628AB91868DA6890420DD2121A83E8A0
:102F70001400202383F311880B482146FFF78AFFB2
:102F800084F31188BDE8F081012303FA04F26B8910
:102F900023EA02036B81CB6823B121460248BDE8D6
:102FA000F0411847BDE8F081B438022000EB8103FE
:102FB0004A0170B5DD68C36E6C692668E66056BB71
:102FC0001A444FF40020C2F810092A6802F00302E4
:102FD000012A0AB20ED1D3F8080803EB421410F408
:102FE000807FD4F8000914BF40F0805040F00050BA
:102FF000C4F8000903EB4212D2F8000940F0044083
:10300000C2F800090122D3F8340802FA01F10143A1
:10301000C3F8341870BD19B9402E84BF4020206019
:1030200020681A442E8A841940F00050013CB4FBF9
:10303000F6F440EAC440C6E7F8B504461E48C56E3B
:1030400005EB4413D3F80869F107C3F8086917D5ED
:10305000D5F81038DA0713D500EB8403D9684B692B
:103060001F68DA68974218D2D21B00271A605F6087
:10307000202383F311882146FFF798FF87F31188F7
:10308000330617D50123D5F83428A340134211D0B5
:103090002046BDE8F840FFF71FBD012303FA04F204
:1030A000038923EA020303818B68002BE8D02146C1
:1030B0009847E5E7F8BD00BFB43802209F482DE9E6
:1030C000F84FC56E04466E69AB691E4016F4805F0A
:1030D0006E6105D0FEF714FDBDE8F84FFFF748BC60
:1030E000002E12DAD5F8003E9B0705D0D5F8003E39
:1030F00023F00303C5F8003ED5F804388F4823F0C9
:103100000103C5F80438FEF727FD370502D58B48C3
:10311000FEF716FDB0040CD5D5F8083813F0060FED
:10312000EB6823F470530CBF43F4105343F4A053E3
:10313000EB60310704D56368DB680BB17F489847C3
:10314000F2026FD4B3020CD5D4F86C8000274FF094
:103150000109DFF8E8A1236FF9B29B688B4280F088
:103160009C80F70619D5E16E0A6AC2F30A1702F0CD
:103170000F0302F4F012B2F5802F00F0B580B2F523
:10318000402F0AD104EB830301F58051DB68186AF4
:1031900000231A469F4240F09C803303D5F818481C
:1031A0001DD5E70302D50020FFF7B2FEA50302D527
:1031B0000120FFF7ADFE600302D50220FFF7A8FE55
:1031C000210302D50320FFF7A3FEE20202D504206B
:1031D000FFF79EFEA30202D50520FFF799FE7703B5
:1031E0007FF57AAFE60702D50020FFF725FFA50798
:1031F00002D50120FFF720FF600702D50220FFF76C
:103200001BFF210702D50320FFF716FFE20602D5B8
:103210000420FFF711FFA3067FF55EAF0520FFF73F
:103220000BFF59E7D4F86C8000274FF00109DFF855
:103230000CA1236F5FFA87FB9B685B4582D308EB89
:103240004B13D3F8002902F44022B2F5802F22D18B
:10325000D3F80029002A1EDAD3F8002942F0904260
:10326000C3F80029D3F80029002AFBDB5946E06E99
:10327000FFF728FC228909FA0BF322EA03032381D2
:1032800004EB8B03DB689B6813B1594650469847A3
:103290005846FFF721FC0137CBE708EB4112D2F883
:1032A000003B03F44023B3F5802F10D1D2F8003B4C
:1032B000002B0CDA628909FA01F322EA0303638125
:1032C00004EB8103DB68DB680BB15046984701379C
:1032D00041E79C0700D10A68072B03F101039EBF59
:1032E0000270120A013055E7023301F5805104EBF8
:1032F0008302526890690268D0F808C04068A2EB67
:10330000000E0022104697420AD104EB8304636842
:103310009B699A683A449A605A6817445F603CE730
:1033200012F0030F00D10868964502F1010282BF36
:103330008CF80000000A0CF1010CE4E7B43802201C
:10334000C36E03EB4111D1F8003B43F40013C1F805
:10335000003B7047C36E03EB4111D1F8003943F4D1
:103360000013C1F800397047C36E03EB4111D1F867
:10337000003B23F40013C1F8003B7047C36E03EB1E
:103380004111D1F8003923F40013C1F80039704716
:1033900030B50433039C0172002104FB0325C36193
:1033A000049B00600363059B4060C1604261026151
:1033B0008561046242628162C162436330BD000084
:1033C0000022416AC260416101616FF001018262C5
:1033D000C262FEF773BF000003694269934203D1E2
:1033E000C2680AB100207047181D70470369196050
:1033F0000021C2680132C260C269134482699342EB
:10340000036124BF436A0361FEF74CBF38B504462D
:103410000D46E3683BB162690020131D1268A36288
:103420001344E36238BD237A33B929462046FEF7B8
:1034300029FF0028EDDA38BD6FF00100FBE700003E
:10344000C368C269013BC360436913448269934204
:10345000436124BF436A436100238362036B03B16A
:103460001847704770B52023044683F31188866A95
:103470003EB9FFF7CBFF054618B186F31188284601
:1034800070BDA36AE26A13F8015B9342A36202D3A0
:103490002046FFF7D5FF002383F31188EFE70000F4
:1034A0002DE9F84F04460E4690469946202787F3AB
:1034B00011880025AA46D4F828B0BBF1000F09D125
:1034C00049462046FFF7A2FF20B18BF3118828461A
:1034D000BDE8F88FA16AA8EB050BE36A5B1A9B4570
:1034E00028BF9B46BBF1400F1BD9334601F1400278
:1034F00051F8040B914243F8040BF9D1A36A40360A
:1035000040354033A362A26AE36A9A4202D320465E
:10351000FFF796FF8AF311884545D8D287F31188C3
:10352000C9E730465A46FDF74DFCA36A5E445D4448
:103530005B44A362E7E7000010B5029C043301720C
:10354000C36103FB0421002300608362C362039B09
:1035500040600363049BC460426102618161046254
:103560004262436310BD0000026A6FF00101C26055
:10357000426A4261026100228262C262FEF79EBE1E
:10358000436902699A4203D1C2680AB100207047B8
:10359000184650F8043B0B6070470000C3680021D8
:1035A000C2690133C3604369134482699342436132
:1035B00024BF436A4361FEF775BE000038B5044678
:1035C0000D46E3683BB1236900201A1DA262E2693F
:1035D0001344E36238BD237A33B929462046FEF707
:1035E00051FE0028EDDA38BD6FF00100FBE7000066
:1035F00003691960C268013AC260C26913448269F2
:103600009342036124BF436A036100238362036B17
:1036100003B118477047000070B5202304460E46DA
:1036200083F31188856A35B91146FFF7C7FF10B1DA
:1036300085F3118870BDA36A1E70A36AE26A013324
:103640009342A36204D3E16920460439FFF7D0FF17
:10365000002080F3118870BD2DE9F84F04460D4617
:1036600091469A464FF0200888F311880026B34609
:10367000A76A4FB951462046FFF7A0FF20B187F354
:1036800011883046BDE8F88FA06AA9EB0603E76A07
:103690003F1A9F4228BF1F46402F1BD905F1400308
:1036A00055F8042B9D4240F8042BF9D1A36A40360B
:1036B0004033A362A26AE36A9A4204D3E1692046D6
:1036C0000439FFF795FF8BF311884E45D9D288F363
:1036D0001188CDE729463A46FDF774FBA36A3D44BD
:1036E0003E443B44A362E5E7026943699A4203D141
:1036F000C3681BB9184670470023FBE7836A002B99
:10370000F8D0043B9B1AF5D01360C368013BC3603B
:10371000C3691A4483699A42026124BF436A036100
:10372000002383620123E5E700F0AEB84FF0804349
:10373000002258631A610222DA60704700224FF0BB
:103740008043DA60704700004FF080435863704751
:103750004B6843608B688360CB68C3600B694361CF
:103760004B6903628B6943620B680360704700001A
:1037700008B5274B40F2FF7126481A690A431A61BF
:103780001A6922F4FF6222F007021A611A691A6BA1
:103790000A431A631A6D0A431A651F4A1B6D1146C4
:1037A000FFF7D6FF1D4802F11C01FFF7D1FF1C48AF
:1037B00002F13801FFF7CCFF1A4802F15401FFF77C
:1037C000C7FF194802F17001FFF7C2FF174802F165
:1037D0008C01FFF7BDFF164802F1A801FFF7B8FF03
:1037E000144802F1C401FFF7B3FF134802F1E001EE
:1037F000FFF7AEFF114802F1FC01FFF7A9FF1048E7
:1038000002F58C71FFF7A4FFBDE8084000F09EB8F8
:103810000038024000000240B83E000800040240A8
:1038200000080240000C0240001002400014024058
:1038300000180240001C0240002002400024024008
:103840000028024008B500F0F5F9FEF73FFCFFF74D
:103850006DF8BDE80840FEF749BE00007047000063
:103860004FF080431A69920710B508D500241C61F7
:10387000202383F31188FEF76DFC84F31188BDE8E3
:103880001040FFF775B80000104B08211C201A6C7F
:1038900042F001021A641A6E42F001021A660C4AE2
:1038A0001B6E936843F0010393604FF080436B22DB
:1038B0009A624FF0FF32DA6200229A615A63DA604C
:1038C0005A6001225A611A60FDF724BD0038024097
:1038D000002004E01B4B4FF0FF3000211A696FEA13
:1038E00042526FEA52521A611A69C2F30A021A610D
:1038F0001A695A6958615A6959615A691A6A62F0B3
:1039000080521A621A6A02F080521A621A6A5A6A5D
:1039100058625A6A59625A6A0B4A106840F48070B9
:103920001060186F00F44070B0F5007F03D04FF4C2
:10393000803018671967536823F40073536000F0F0
:1039400059B900BF0038024000700040354B4FF4B9
:103950004041354A1A64354A11601A6842F0010242
:103960001A601A689207FCD59A6822F003029A60DE
:103970002C4B19469A6812F00C02FBD1186800F023
:10398000F90018609A601A6842F480321A600B6875
:103990009B03FCD54B6F43F001034B67214B5A6FE0
:1039A0009007FCD5224A5A601A6842F080721A6069
:1039B0001E4B1A4659684904FCD5196841F48031F8
:1039C00019605368D803FCD5136843F400331360BF
:1039D000164A53689903FCD5124B1A689201FCD51C
:1039E000144A40F207319A6040F20112C3F88C2069
:1039F0000022C3F89020104A11609A6842F0020237
:103A00009A60084B9A6802F00C02082AFAD15A6CA4
:103A100042F480425A645A6E42F480425A665B6EA7
:103A2000704700BF003802400004001000700040E2
:103A30000836400900948838003C0240084A08B51E
:103A4000536911680B4003F00103536123B1054A28
:103A500013680BB150689847BDE80840FEF788BF6F
:103A6000003C0140C8250220084A08B55369116886
:103A70000B4003F00203536123B1054A93680BB175
:103A8000D0689847BDE80840FEF772BF003C01408F
:103A9000C8250220084A08B5536911680B4003F095
:103AA0000403536123B1054A13690BB15069984768
:103AB000BDE80840FEF75CBF003C0140C82502207D
:103AC000084A08B5536911680B4003F008035361B5
:103AD00023B1054A93690BB1D0699847BDE8084006
:103AE000FEF746BF003C0140C8250220084A08B541
:103AF000536911680B4003F01003536123B1054A69
:103B0000136A0BB1506A9847BDE80840FEF730BF12
:103B1000003C0140C8250220174B10B55C691A68AB
:103B2000144004F478725A61A30604D5134A936AC8
:103B30000BB1D06A9847600604D5104A136B0BB1DD
:103B4000506B9847210604D50C4A936B0BB1D06B90
:103B50009847E20504D5094A136C0BB1506C98479D
:103B6000A30504D5054A936C0BB1D06C9847BDE80A
:103B70001040FEF7FDBE00BF003C0140C8250220FA
:103B80001A4B10B55C691A68144004F47C425A61FF
:103B9000620504D5164A136D0BB1506D9847230585
:103BA00004D5134A936D0BB1D06D9847E00404D54A
:103BB0000F4A136E0BB1506E9847A10404D50C4AFE
:103BC000936E0BB1D06E9847620404D5084A136F08
:103BD0000BB1506F9847230404D5054A936F0BB17E
:103BE000D06F9847BDE81040FEF7C2BE003C0140D0
:103BF000C8250220062108B50846FDF78BFB0621E3
:103C00000720FDF787FB06210820FDF783FB06212F
:103C10000920FDF77FFB06210A20FDF77BFB06212B
:103C20001720FDF777FB06212820BDE80840FDF7A7
:103C300071BB000008B5FFF74DFEFDF7FDF9FDF77C
:103C400013FDFDF7E9FEFDF7BDFDFFF707FEBDE83B
:103C50000840FFF769BD0000034611F8012B03F887
:103C6000012B002AF9D17047121012131211000013
:103C70000010410001105A0058310220482602204D
:103C8000B426022053544D3332463F3F3F3F3F3F1F
:103C90000053544D333246375B347C355D780053E6
:103CA000544D333246375B367C375D780000000078
:103CB000009600000000000000000000000000006E
:103CC00000000000000000000000000031160008A5
:103CD0001D16000859160008451600085116000860
:103CE0003D1600082916000815160008651600087C
:103CF000000000003D17000829170008651700089C
:103D0000511700085D17000849170008351700080B
:103D100021170008C1170008000000000100000082
:103D2000000000006D61696E00000000443D000865
:103D3000602F02205831022001000000C920000835
:103D40000000000069646C650000000002000000D3
:103D50000000000069190008D11900084000400067
:103D6000F0350220003602200200000000000000B2
:103D70000300000000000000151A00080000000009
:103D800010000000103602200000000001000000BA
:103D900000000000B438022001010200486F6C7975
:103DA00062726F00706978333276352D424C00258F
:103DB00053455249414C25008D240008F523000845
:103DC000D51800087124000843000000D03D000809
:103DD00009024300020100C032090400000102028E
:103DE0000100052400100105240100010424020241
:103DF0000524060001070582030800FF09040100ED
:103E0000020A0000000705010240000007058102C8
:103E100040000000120000001C3E000812011001CA
:103E20000200004062314E00000201020301000066
:103E30000403090425424F41524425005069783358
:103E40003276350030313233343536373839414205
:103E50004344454600000000008000000080000050
:103E6000008000000080000000000200000004004C
:103E70000000040000000400000004000000040032
:103E80000000040000000400000000006D1B00089A
:103E90004D1E0008F91E0008400040002C39022089
:103EA0002C390220010000003C3902208000000073
:103EB00040010000050000000000802A0000000012
:103EC000AAAAAAAA00000000FFFF0000000000004C
:103ED00000A00A000000000000000000AAAAAAAA90
:103EE00000000000FFFF00000000000000000000D4
:103EF0000050000000000000AAAAAAAA00000000CA
:103F0000FFFF00000000000000000000802900000A
:103F100000000000AAAAAAAA40150000FFFF0000A6
:103F200000707007000000000000020000000000A8
:103F3000AAAAAAAA00000100FFFF000000000000DA
:103F40000800000050255000000000000AA2AAAAA4
:103F500050155000FFFF00000000000800000000A6
:103F60000000100000000000AAAAAAAA0000100089
:103F7000FFFF00000000000000000000000400003F
:103F800000000000AAAAAAAA00040000FFFF000087
:103F9000000000000000000000515100000000007F
:103FA000AAAAAAAA00515100FFFF000000000000C9
:103FB0000000000000000000000000000000000001
:103FC00000000000000000000000000000000000F1
:103FD00000000000000000000000000000000000E1
:103FE00000000000000000000000000000000000D1
:103FF000FF00000000000000843C00083F000000BB
:1040000049040000913C00083F00000051040000FA
:104010009F3C00083F0000000096000000000800E0
:1040200004000000303E0008000000000000000016
:104030000000000000000000000000000000000080
:00000001FF
